:100000000C946C000C9494000C9494000C94940048
:100010000C9494000C9494000C9494000C94940010
:100020000C9494000C9494000C9494000C94940000
:100030000C9494000C9494000C9494000C949400F0
:100040000C94F1060C9494000C94BF060C94990641
:100050000C9494000C9494000C9494000C949400D0
:100060000C943B070C94940000000000240027002F
:100070002A0000000000250028002B0000000008D6
:10008000000201000003040700000000000000005F
:1000900043200054656D703A200048756D656461B9
:1000A000643A200000000000230026002900040418
:1000B0000404040404040202020202020303030310
:1000C00003030102040810204080010204081020EC
:1000D0000102040810205A0811241FBECFEFD8E0F7
:1000E000DEBFCDBF11E0A0E0B1E0E2E5FBE102C080
:1000F00005900D92A634B107D9F722E0A6E4B1E04D
:1001000001C01D92AC3CB207E1F710E0CCE6D0E0B4
:1001100004C02197FE010E94A10DCB36D107C9F77B
:100120000E94C2080C94A70D0C940000CF92DF929D
:10013000EF92FF92CF93DF93B091B302A0E08111D1
:10014000AB2F8091B40290E0880F991FAC014C5501
:100150005F4FC090B902D090BA02E090BB02F0901D
:10016000BC0230E020E0FA01C591D491E881B901E8
:1001700090E080E0EB23EA130AC02F5F3F4F6C153D
:100180007D058E059F0578F36FEF7FEFCB01DF9143
:10019000CF91FF90EF90DF90CF900895089508954C
:1001A000EF92FF920F931F93CF93DF938C017B010C
:1001B000D0E0C0E0F701EC0FFD1F6491662361F011
:1001C000D801ED91FC910190F081E02DC8010995D5
:1001D000892B11F02196EECFCE01DF91CF911F91A7
:1001E0000F91FF90EF900895AF92BF92CF92DF9260
:1001F000EF92FF920F931F93CF93DF936C017B01DC
:100200008B01040F151FEB015E01AE18BF08C0176C
:10021000D10759F06991D601ED91FC910190F081DF
:10022000E02DC6010995892B79F7C501DF91CF91A2
:100230001F910F91FF90EF90DF90CF90BF90AF9004
:100240000895FC01538D448D252F30E0842F90E0DC
:10025000821B930B541710F0CF96089501970895C1
:10026000FC01918D828D981761F0A28DAE0FBF2F8A
:10027000B11D5D968C91928D9F5F9F73928F90E0E0
:1002800008958FEF9FEF0895FC01918D828D98174F
:1002900031F0828DE80FF11D858D90E008958FEF8C
:1002A0009FEF0895FC01918D228D892F90E0805C55
:1002B0009F4F821B91098F739927089583E092E0E5
:1002C0000E94520121E0892B09F420E0822F089539
:1002D00080E090E0892B29F00E945E0181110C944E
:1002E00000000895FC01A48DA80FB92FB11DA35AD9
:1002F000BF4F2C91848D90E001968F739927848F46
:10030000A689B7892C93A089B1898C918370806468
:100310008C93938D848D981306C00288F389E02D09
:1003200080818F7D80830895EF92FF920F931F93BA
:10033000CF93DF93EC0181E0888F9B8D8C8D981398
:100340001AC0E889F989808185FF15C09FB7F894A4
:10035000EE89FF896083E889F989808183708064F0
:1003600080839FBF81E090E0DF91CF911F910F913B
:10037000FF90EF900895F62E0B8D10E00F5F1F4F4A
:100380000F731127E02E8C8D8E110CC00FB607FC59
:10039000FACFE889F989808185FFF5CFCE010E94E7
:1003A0007201F1CFEB8DEC0FFD2FF11DE35AFF4FE2
:1003B000F0829FB7F8940B8FEA89FB898081806275
:1003C000CFCFCF93DF93EC01888D8823B9F0AA8932
:1003D000BB89E889F9898C9185FD03C0808186FD00
:1003E0000DC00FB607FCF7CF8C9185FFF2CF80814F
:1003F00085FFEDCFCE010E947201E9CFDF91CF9151
:10040000089590E0FC01E458FF4F2491FC01EE5365
:10041000FF4F3491FC01E255FF4FE491EE23C9F008
:10042000222339F0233001F1A8F4213019F12230D0
:1004300029F1F0E0EE0FFF1FEE58FF4FA591B491A8
:100440008FB7F894EC91611126C030953E233C9310
:100450008FBF08952730A9F02830C9F0243049F71C
:10046000809180008F7D03C0809180008F77809382
:100470008000DFCF84B58F7784BDDBCF84B58F7DDF
:10048000FBCF8091B0008F778093B000D2CF809166
:10049000B0008F7DF9CF3E2BDACFCF93DF9390E082
:1004A000FC01EE53FF4F249182559F4FFC01849134
:1004B0008823D1F090E0880F991FFC01E859FF4F85
:1004C000A591B491FC01EE58FF4FC591D4916230D3
:1004D00071F49FB7F8943C91822F809583238C937D
:1004E000E8812E2B28839FBFDF91CF9108958FB78E
:1004F000F894EC912E2B2C938FBFF6CF3FB7F89446
:100500008091F0019091F101A091F201B091F3017D
:1005100026B5A89B05C02F3F19F00196A11DB11D5E
:100520003FBFBA2FA92F982F8827BC01CD01620F9A
:10053000711D811D911D42E0660F771F881F991F55
:100540004A95D1F708958F929F92AF92BF92CF9222
:10055000DF92EF92FF924B015C010E947E026B01E1
:100560007C010E947E026C197D098E099F09683EFC
:10057000734081059105A8F321E0821A9108A10832
:10058000B10888EEC80E83E0D81EE11CF11C81146E
:100590009104A104B10429F7FF90EF90DF90CF9070
:1005A000BF90AF909F908F900895CF92DF92EF927F
:1005B000FF920F931F93CF93DF93CDB7DEB7C05455
:1005C000D1400FB6F894DEBF0FBECDBF2FB7F89461
:1005D0008091FF0190910002A0910102B09102026E
:1005E0002FBF4091B5025091B6026091B702709151
:1005F000B8028C019D01041B150B260B370BB901AA
:10060000A801403D57406105710590F48091BD02FD
:10061000C05CDE4F0FB6F894DEBF0FBECDBFDF91DA
:10062000CF911F910F91FF90EF90DF90CF900895A1
:100630008093B5029093B602A093B702B093B8022C
:100640001092B0021092AF021092AE021092AD0260
:100650001092AC0262E08091B1020E944D0261E012
:1006600070E080E090E00E94A30261E08091B1021E
:100670000E944D0260E08091B1020E9401028091CF
:10068000B2028551823020F58BE291E10197F1F7BA
:1006900062E08091B1020E944D028091BE0290E022
:1006A0008230910538F0880F991F880F991F0597A0
:1006B0000197F1F7F89480E00E9496006F3F7F4F1A
:1006C0008F4F9F4F61F41092BD02789480E0A0CFCD
:1006D00064E170E080E090E00E94A302D9CF81E065
:1006E0000E9496006F3F7F4F8F4F9F4F61F38E01A7
:1006F0000F5F1F4F6E018FEBC81A8EEFD80A78017B
:1007000080E00E949600F701608371838283938367
:1007100081E00E949600F701648375838683978346
:10072000F8E0EF0EF11CEC14FD0451F7789430E082
:1007300020E0F801C080D180E280F38044815581BF
:1007400066817781FFEFCF16DF06EF06FF0631F0F7
:100750004F3F8FEF58076807780719F41092BD02D2
:10076000B5CFF90183E0F595E7958A95E1F7E45572
:10077000FD4F8081880FC416D506E606F70610F1F6
:1007800080832F5F3F4F085F1F4F2832310589F666
:100790004091B0022091AC028091AD02280F332726
:1007A000331F8091AE02280F311D8091AF02820F5E
:1007B000932F911D99274817190681F681E08093A0
:1007C000BD0226CF8160DCCF089585ED8093BC000B
:1007D0008091BC0084FDFCCF1092FA010895209115
:1007E0008601260F3327331F21323105ECF4209187
:1007F000FA01FC0190E080E0243069F082E0089585
:10080000A09186012191AC014A595E4FA40FB52FEA
:10081000B11D2C930196861798F380918601680F7D
:100820006093860180E0089581E008950895E09145
:10083000FE018091FD01E81730F4F0E0EA5BFE4F25
:10084000808190E008958FEF9FEF08959091FE01D1
:100850008091FD012FEF3FEF981748F4E92FF0E06A
:10086000EA5BFE4F208130E09F5F9093FE01C9015B
:1008700008958091FD019091FE01891B990B0895C7
:10088000CF92DF92EF92FF920F931F93CF93DF935C
:100890007C01CB018A012091CD01222389F0EB015B
:1008A0006B01C40ED51ECC15DD0569F06991D70129
:1008B000ED91FC910190F081E02DC7010995F3CFF6
:1008C000642F0E94EF03C801DF91CF911F910F9118
:1008D000FF90EF90DF90CF900895CF93DF931F921A
:1008E000CDB7DEB769832091CD012223F9F02091A5
:1008F000FB01203258F021E030E0FC0133832283F9
:1009000090E080E00F90DF91CF9108958091FC01FD
:10091000E82FF0E0E253FE4F998190838F5F809340
:10092000FC018093FB0181E090E0ECCF61E0CE011F
:1009300001960E94EF03F7CFCF93FC01C48121E021
:100940002093CD01C093EE011092FC011092FB01A7
:100950008485682B80EA92E00E946D049091FB01EF
:10096000913208F03FC08091FA018111FCCF82E002
:100970008093FA0181E08093F9018FEF8093CC019D
:100980001092CB019093CA01AEECB1E0EAEAF1E03B
:1009900080E098132FC01092A9018091A901CC0F7B
:1009A000C82BC093A9018091F801813039F51092CC
:1009B000F8018091A9018093BB008091BC0083FD68
:1009C000F8CF85EC8093BC008091FA018230E1F38E
:1009D0008091CC018F3F31F08091CC01803211F0B9
:1009E0008091CC011092FC011092FB011092CD017C
:1009F000CF9108952D9121938F5FCBCF85EEE2CFDC
:100A000090E080E00895FC0101900020E9F7319723
:100A1000AF01481B590BBC018FEB92E00C94F40022
:100A20008F929F92AF92BF920F931F93CF93DF93BA
:100A3000CDB7DEB7A1970FB6F894DEBF0FBECDBF1E
:100A400019A2423008F44AE08E010F5D1F4F842E38
:100A5000912CB12CA12CA50194010E947F0DE62FB1
:100A6000B901CA01EA30F4F4E05DD801EE938D01DA
:100A7000232B242B252B79F790E080E0109719F099
:100A8000CD010E940305A1960FB6F894DEBF0FBEFC
:100A9000CDBFDF91CF911F910F91BF90AF909F90ED
:100AA0008F900895E95CE1CF0F931F93CF938C0152
:100AB000C62F0E949C046C2F6460C8010E949C0495
:100AC0006C2F6B7FC8010E949C0483EC90E001971F
:100AD000F1F7CF911F910F9108950F931F93CF932B
:100AE000DF938C01D62FC42F607F642B0E945405A6
:100AF00080E1D89FB00111246C2BC801DF91CF9108
:100B00001F910F910C945405CF93DF93CDB7DEB7AF
:100B100028970FB6F894DEBF0FBECDBF98E0E0E097
:100B2000F1E0DE01119601900D929A95E1F7909116
:100B3000C702981708F48FEF90E0880F991F21E003
:100B400030E02C0F3D1F820F931FFC016081606815
:100B500040E08FEB92E028960FB6F894DEBF0FBE10
:100B6000CDBFDF91CF910C946D0541E00E946D05E2
:100B700081E090E008954F925F926F927F928F9202
:100B80009F92AF92BF92CF92DF92EF92FF920F931C
:100B90001F93CF936B017C01742EAC019B010E94CB
:100BA0007A0D882399F088E391E0CF911F910F91FE
:100BB000FF90EF90DF90CF90BF90AF909F908F907D
:100BC0007F906F905F904F900C9403054601570102
:100BD000E894B7F82FEF3FEF4FE75FE7C501B401A7
:100BE0000E947A0D81110DC02FEF3FEF4FE75FE7B5
:100BF000C501B4010E94B00B18161CF48CE391E0FF
:100C0000D4CF2FEF3FEF4FE75FE4C701B6010E945B
:100C1000080D18161CF480E491E0C7CF2FEF3FEFCA
:100C20004FE75FECC701B6010E94B00B87FDF3CF21
:100C300020E030E0A901C701B6010E94B00B10E02E
:100C400000E087FF0CC041E06DE28FEB92E00E9474
:100C50006D05F7FAF094F7F8F09401E010E0C0E0C9
:100C600060E070E080E09FE37C1641F020E030E03F
:100C700040E251E40E94B50BCF5FF6CFA701960189
:100C80000E94440B4B015C010E94270C2B013C018C
:100C90004AE00E941005080F191FCC23C9F1C301B7
:100CA000B2010E94560C9B01AC01C501B4010E9427
:100CB000430B4B015C0141E06EE28FEB92E00E943E
:100CC0006D050F5F1F4FC15018F120E030E040E28A
:100CD00051E4C501B4010E940D0D2B013C010E949D
:100CE000270C4B01B12CA12C4AE0C501B4010E9494
:100CF0001005080F191FC501B4010E94560C9B0175
:100D0000AC01C301B2010E94430B4B015C01DBCF7C
:100D1000C801CF911F910F91FF90EF90DF90CF907E
:100D2000BF90AF909F908F907F906F905F904F900B
:100D300008951F920F920FB60F9211242F933F9395
:100D40004F935F936F937F938F939F93AF93BF93D3
:100D5000EF93FF9383E092E00E947201FF91EF9185
:100D6000BF91AF919F918F917F916F915F914F91C3
:100D70003F912F910F900FBE0F901F9018951F92CB
:100D80000F920FB60F9211242F938F939F93EF938F
:100D9000FF93E0911302F09114028081E091190217
:100DA000F0911A0282FD1BC0908180911C028F5F1E
:100DB0008F7320911D02821741F0E0911C02F0E038
:100DC000ED5FFD4F958F80931C02FF91EF919F91F6
:100DD0008F912F910F900FBE0F901F9018958081CB
:100DE000F4CF1F920F920FB60F9211242F933F93BF
:100DF0008F939F93AF93BF938091FF0190910002D7
:100E0000A0910102B09102023091EF0123E0230F83
:100E10002D3758F50196A11DB11D2093EF01809348
:100E2000FF0190930002A0930102B093020280910F
:100E3000F0019091F101A091F201B091F3010196BE
:100E4000A11DB11D8093F0019093F101A093F201D7
:100E5000B093F301BF91AF919F918F913F912F91EB
:100E60000F900FBE0F901F90189526E8230F029643
:100E7000A11DB11DD2CF1F920F920FB60F92112458
:100E80002F933F934F935F936F937F938F939F9392
:100E9000AF93BF93EF93FF938091B900887F803623
:100EA00009F44AC0F0F5883209F4A7C018F580317A
:100EB00009F49BC0B8F4882309F4F9C0883009F418
:100EC00094C0FF91EF91BF91AF919F918F917F91CE
:100ED0006F915F914F913F912F910F900FBE0F90A7
:100EE0001F901895883109F488C0803251F780939B
:100EF000CC0114C0803409F49DC040F48033B9F3B0
:100F00008833F9F68093CC0185ECB0C0803509F4C4
:100F100085C0883509F496C0883499F60E94E503A7
:100F2000D0CF883909F48CC038F5883729F050F4CF
:100F3000883611F0803729F683E08093FA01109209
:100F4000A80157C0883809F47BC0803919F080386F
:100F500009F0B7CF8091A801803208F071C0E0910C
:100F6000A80181E08E0F8093A8018091BB00F0E082
:100F7000E857FE4F80833DC0803B39F0E0F4803A73
:100F800009F479C0883A09F09CCF84E08093FA0193
:100F90001092870110928601E091F601F091F7011D
:100FA00009958091860181110FC081E080938601AF
:100FB0001092660109C0803C09F4A6CF883C09F470
:100FC000A3CF883B09F07DCFE091870181E08E0FB0
:100FD00080938701F0E0EA59FE4F80818093BB0047
:100FE000909187018091860129C08091A901809309
:100FF000BB0085EC8093BC0064CF9091CB018091C5
:10100000CA01981758F5E091CB0181E08E0F8093CB
:10101000CB01F0E0E655FE4F8081E9CFE091CB01B6
:1010200081E08E0F8093CB018091BB00F0E0E6550C
:10103000FE4F80839091CB018091CA019817C8F22E
:1010400085E8D8CFE091CB0181E08E0F8093CB0172
:101050008091BB00F0E0E655FE4F80838091F9015E
:1010600081115CCF81E08093F80184EA8093BC0019
:101070001092FA0126CF85EC8093BC001092FA0101
:101080008091A801803230F4E091A801F0E0E857A7
:10109000FE4F10826091A80170E0E091F401F091A0
:1010A000F50188E891E009951092A8010ACF109205
:1010B000CC0134CFE3E0F2E01382128288EE93E0B9
:1010C000A0E0B0E084839583A683B7832CE031E071
:1010D0003183208325EC30E03587248724EC30E011
:1010E0003787268720EC30E0318B208B21EC30E0F5
:1010F000338B228B22EC30E0358B248B26EC30E0D6
:10110000378B268B118E128E138E148EE0EAF2E04E
:101110001382128284839583A683B7838EE191E044
:1011200091838083EFEBF2E01382128280E391E0FF
:101130009183808311868FE3848380E1828782E0BC
:1011400083871486ACEAB2E015968C9315978BE0F2
:1011500016968C931697E4ECF0E0E4911796EC93D6
:101160001797E0EBF0E0E4911896EC93189740E8BD
:101170005EE360E070E01D964D935D936D937C930C
:1011800050970895789484B5826084BD84B5816059
:1011900084BD85B5826085BD85B5816085BD809142
:1011A0006E00816080936E001092810080918100BA
:1011B00082608093810080918100816080938100B2
:1011C000809180008160809380008091B100846074
:1011D0008093B1008091B00081608093B0008091D5
:1011E0007A00846080937A0080917A008260809394
:1011F0007A0080917A00816080937A0080917A00F1
:10120000806880937A001092C10061E087E00E94BC
:101210004D0261E085E00E944D0261E086E00E949F
:101220004D02E0911302F091140282E08083E0917C
:101230000F02F09110021082E0911102F09112025F
:101240008FEC808310921B02E0911702F09118023C
:1012500086E08083E0911502F09116028081806122
:101260008083E0911502F09116028081886080836E
:10127000E0911502F0911602808180688083E091F0
:101280001502F091160280818F7D808362E080914B
:10129000B1020E944D022FB7F8948091FF01909106
:1012A0000002A0910102B09102022FBF805D974021
:1012B000A109B1098093B5029093B602A093B70239
:1012C000B093B80287E38093BE021092FE011092A1
:1012D000FD011092FC011092FB011092FA0181E0D5
:1012E0008093F9011092F80161E082E10E9401020D
:1012F00061E083E10E9401028091B9008E7F8093BA
:10130000B9008091B9008D7F8093B90088E4809303
:10131000B80085E48093BC008EEC90E09093F701D8
:101320008093F6018FEC90E09093F5018093F401A7
:101330001092C4028091CA02823018F098E0909313
:10134000C4028093C70262E370E080E090E00E94F4
:10135000A3026091CB028FEB92E00E949C0468EEA6
:1013600073E080E090E00E94A30260E38FEB92E0E4
:101370000E945405CBE4D6E4CE010197F1F760E377
:101380008FEB92E00E9454052197F1F760E38FEB19
:1013900092E00E94540583E592E00197F1F760E244
:1013A0008FEB92E00E9454056091C402606240E0BD
:1013B0008FEB92E00E946D0584E08093C50240E0CF
:1013C0006CE08FEB92E00E946D0540E061E08FEBF6
:1013D00092E00E946D058BE39FE10197F1F7809108
:1013E000C802882319F080E00E94840582E080937F
:1013F000C60240E066E08FEB92E00E946D0540E09F
:1014000062E08FEB92E00E946D058BE39FE1019714
:10141000F1F788E08093CB0260E08FEB92E00E94CE
:101420009C04C0E0D0E060ED77E080E090E00E94B6
:10143000A3020E94D502882349F08091B2028B302A
:1014400028F08D3050F085518230C0F1812C912CE4
:1014500020ECA22E2FE7B22E1EC06091AD0270E0EC
:1014600090E080E00E94580C2DEC3CEC4CEC5DE3ED
:101470000E940D0D6B017C016091AC0270E090E068
:1014800080E00E94580C9B01AC01C701B6010E948C
:10149000440B4B015C010E94D502882341F08091EE
:1014A000B2028C3009F4A6C0D8F48B3091F1C12C73
:1014B000D12C80ECE82E8FE7F82E55C06091AC025D
:1014C0007091AD0276276727762790E080E00E9432
:1014D000560C2DEC3CEC4CEC5DE30E940D0DD9CF8D
:1014E0008551823020F71091AE02612F70E0762F87
:1014F000662766277F778091AF02682B90E080E0B7
:101500000E94560C2DEC3CEC4CEC5DE30E940D0D62
:101510008DC06091AE0270E090E080E00E94560CB9
:101520006B017C011091AF0217FF0AC0AC019B0157
:1015300060E070E080E89FEB0E94430B6B017C0150
:101540001F70612F70E090E080E00E94580C2DEC3D
:101550003CEC4CEC5DE30E940D0DA70196010E944E
:10156000440B6B017C0180E00E9484056AE970E015
:101570008FEB92E00E94D00042E0C501B4010E94CE
:10158000BB0584E491E00E94030581E00E9484058C
:1015900063E970E08FEB92E00E94D00042E0C70167
:1015A000B6010E94BB0560E970E083E092E00E9412
:1015B000D00020E030E040EE51E4C701B6010E94C7
:1015C000080D87FD3CC061E087E00E94010260E0F9
:1015D00085E00E94010260E086E00E9401022097FF
:1015E00009F421CF0E945E01882309F41CCF0E94D8
:1015F000000019CF1091AE02612F70E090E080E002
:101600000E94560C6B017C016091AF026F7070E01C
:1016100090E080E00E94580C2DEC3CEC4CEC5DE33B
:101620000E940D0DA70196010E94440B6B017C01E5
:1016300017FF99CFF7FAF094F7F8F09494CF20E0E1
:1016400030E040EA51E4C701B6010E94080D87FD71
:1016500010C020E030E040ED51E4C701B6010E9427
:10166000B00B181634F060E087E00E94010261E0E0
:10167000AFCF60E087E00E94010260E085E00E9459
:10168000010261E0A9CF5058BB27AA270E945B0B3B
:101690000C94CE0C0E94C00C38F00E94C70C20F0B5
:1016A00039F49F3F19F426F40C94BD0C0EF4E09528
:1016B000E7FB0C94B70CE92F0E94DF0C58F3BA1724
:1016C000620773078407950720F079F4A6F50C9458
:1016D000010D0EF4E0950B2EBA2FA02D0B01B901D0
:1016E00090010C01CA01A0011124FF27591B99F098
:1016F000593F50F4503E68F11A16F040A22F232FA4
:10170000342F4427585FF3CF469537952795A795F3
:10171000F0405395C9F77EF41F16BA0B620B730B9A
:10172000840BBAF09150A1F0FF0FBB1F661F771F0B
:10173000881FC2F70EC0BA0F621F731F841F48F4C0
:10174000879577956795B795F7959E3F08F0B0CF49
:101750009395880F08F09927EE0F97958795089530
:101760000E94930C08F481E008950E94C90B0C9428
:10177000CE0C0E94C70C58F00E94C00C40F029F417
:101780005F3F29F00C94B70C51110C94020D0C948E
:10179000BD0C0E94DF0C68F39923B1F3552391F33C
:1017A000951B550BBB27AA2762177307840738F0D0
:1017B0009F5F5F4F220F331F441FAA1FA9F335D02D
:1017C0000E2E3AF0E0E832D091505040E695001CE1
:1017D000CAF72BD0FE2F29D0660F771F881FBB1F9B
:1017E000261737074807AB07B0E809F0BB0B802D79
:1017F000BF01FF2793585F4F3AF09E3F510578F0A5
:101800000C94B70C0C94020D5F3FE4F3983ED4F3B4
:10181000869577956795B795F7959F5FC9F7880F78
:10182000911D9695879597F90895E1E0660F771FCA
:10183000881FBB1F621773078407BA0720F0621B5B
:10184000730B840BBA0BEE1F88F7E09508950E9486
:10185000E70C88F09F5798F0B92F9927B751B0F04F
:10186000E1F0660F771F881F991F1AF0BA95C9F724
:1018700014C0B13091F00E94010DB1E008950C94B4
:10188000010D672F782F8827B85F39F0B93FCCF367
:10189000869577956795B395D9F73EF490958095A1
:1018A000709561957F4F8F4F9F4F0895E89409C0C1
:1018B00097FB3EF490958095709561957F4F8F4F83
:1018C0009F4F9923A9F0F92F96E9BB279395F69599
:1018D000879577956795B795F111F8CFFAF4BB0F17
:1018E00011F460FF1BC06F5F7F4F8F4F9F4F16C07B
:1018F000882311F096E911C0772321F09EE8872F05
:10190000762F05C0662371F096E8862F70E060E0C0
:101910002AF09A95660F771F881FDAF7880F969539
:10192000879597F90895990F0008550FAA0BE0E8DD
:10193000FEEF16161706E807F907C0F01216130691
:10194000E407F50798F0621B730B840B950B39F4D1
:101950000A2661F0232B242B252B21F408950A2637
:1019600009F4A140A6958FEF811D811D089597F977
:101970009F6780E870E060E008959FEF80EC089535
:1019800000240A941616170618060906089500245E
:101990000A9412161306140605060895092E0394D8
:1019A000000C11F4882352F0BB0F40F4BF2B11F44C
:1019B00060FF04C06F5F7F4F8F4F9F4F089557FDAB
:1019C0009058440F551F59F05F3F71F04795880FAD
:1019D00097FB991F61F09F3F79F087950895121644
:1019E00013061406551FF2CF4695F1DF08C01616F0
:1019F00017061806991FF1CF8695710561050894A1
:101A00000895E894BB2766277727CB0197F90895B7
:101A10000E94930C08F48FEF08950E94200D0C94FF
:101A2000CE0C0E94C00C38F00E94C70C20F0952309
:101A300011F00C94B70C0C94BD0C11240C94020DF5
:101A40000E94DF0C70F3959FC1F3950F50E0551F76
:101A5000629FF001729FBB27F00DB11D639FAA2703
:101A6000F00DB11DAA1F649F6627B00DA11D661F52
:101A7000829F2227B00DA11D621F739FB00DA11D73
:101A8000621F839FA00D611D221F749F3327A00D2D
:101A9000611D231F849F600D211D822F762F6A2FC9
:101AA00011249F5750409AF0F1F088234AF0EE0F2E
:101AB000FF1FBB1F661F771F881F91505040A9F75B
:101AC0009E3F510580F00C94B70C0C94020D5F3FC3
:101AD000E4F3983ED4F3869577956795B795F79597
:101AE000E7959F5FC1F7FE2B880F911D969587950F
:101AF00097F908950E94930C880B990B0895A1E221
:101B00001A2EAA1BBB1BFD010DC0AA1FBB1FEE1F77
:101B1000FF1FA217B307E407F50720F0A21BB30BC2
:101B2000E40BF50B661F771F881F991F1A9469F73E
:101B300060957095809590959B01AC01BD01CF019A
:101B40000895EE0FFF1F0590F491E02D0994F8948D
:021B5000FFCFC5
:101B52000000400014005400000000009401F40052
:101B62002101E101520130014401000000006D0435
:101B7200400400051604390426041704000000007E
:101B8200B505F4000005E4036E616E00696E66003F
:061B92006F7666002500DD
:00000001FF
